:107000000C942A380C9437390C9445380C94453834
:107010000C9445380C9445380C9445380C944538FC
:107020000C9445380C9445380C9445380C944538EC
:107030000C9445380C9445380C9445380C944538DC
:107040000C9445380C9445380C9445380C944538CC
:107050000C94453811241FBECFE5D8E0DEBFCDBF6C
:1070600010E0A0E6B0E0E8EFF8E702C005900D926E
:10707000A63AB107D9F711E0A6EAB0E001C01D9227
:10708000A435B107E1F70C94BE380C94003808958C
:1070900008950895AC0120E030E0E0EAFFE005C08B
:1070A000CF010197F1F72F5F3F4F24173507C4F346
:1070B00008951F931FB7F894E199FECFF7E0660F8C
:1070C000771F881F991FFA95D1F783E0FB01809302
:1070D0005700E89507B600FCFDCFAB01AAEBB0E086
:1070E00031E02C91FD0181819927982F8827820F0B
:1070F000911D0C01FA0130935700E8951124129666
:107100004E5F5F4FF1E0AA33BF0759F785E0FB01FF
:1071100080935700E89507B600FCFDCF81E180938E
:107120005700E8951FBF1F91089580E0A0E0B0E0F0
:10713000082E0E94703C8091A900882351F0609134
:10714000AD0066956093AD007727882799270E9448
:10715000593868E08FE20E94773B61E08FE20E943D
:10716000773B61E080E00E94773B81E08BBF1BBEF4
:10717000E091A600F091A70009950895CFE5D8E029
:10718000DEBFCDBFA0E0B0E00E94683C902DF89437
:1071900081E08BBF82E08BBF7894992311F40E9429
:1071A000953888EC90E00E944A3860E670E089E704
:1071B00090E00E94883B86EE98E30E94913B0E94FB
:1071C000463B0E94BC3B1092A900FFCFFC0180917E
:1071D000AA00823041F0853009F448C08130B9F509
:1071E0000E94953808952091AD00822F992780FF45
:1071F0001FC01092A900213019F41092A80007C0F6
:10720000019762E070E00E94413C6093A800DF01BA
:10721000EAEFF0E08D91819381E0EA33F807D1F74E
:107220006091A8007727882799270E9459380CC0B9
:1072300081E08093A900DF01EAEBF0E08D9181937A
:1072400080E0EA3FF807D1F71092AA000895808104
:107250008093AA00823021F481818093AD0008954B
:10726000813021F40E9495381092AA0008951F924F
:107270000F920FB60F9211242F933F934F935F936A
:107280006F937F938F939F93AF93BF93EF93FF93EE
:107290000E94963BFF91EF91BF91AF919F918F918B
:1072A0007F916F915F914F913F912F910F900FBE02
:1072B0000F901F90189587E280933B0185E28093A1
:1072C0003A0190E290933C0110923D0128E030E0B9
:1072D00030933F0120933E0183E28093470181E296
:1072E00080934601909348011092490130934B01DD
:1072F00020934A010895089568E08FE20E94773B49
:1073000062E18CE20E94773B61E08FE20E94773B72
:1073100008950F931F93CF93DF93EC012885398550
:1073200012161306DCF58E819F81821793071CF5D8
:1073300068E083E20E94773B00E010E00FC08A859E
:107340009B85E80FF91F608181E20E94773B8E8167
:107350009F8101969F838E830F5F1F4FEE81FF8178
:1073600088859985083011051CF4E817F9073CF366
:10737000E817F90724F061E087E20E94773B8B81F0
:10738000813031F465E089810E94773B1B8206C021
:1073900061E089810E94773B81E08B83DF91CF910F
:1073A0001F910F910895DC01FC01938110924D0112
:1073B00010924C0181E080934901913019F0923094
:1073C00059F51BC0E091B600F091B7008081992774
:1073D00090934F0180934E01F0935101E09350013F
:1073E000FD018681978180349105B1F488E090E0B9
:1073F00090934F0180934E010FC0FD0186819781CC
:1074000090934F0180934E018091B8009091B90004
:10741000909351018093500186E491E00E94893954
:107420000895CF93DF9382E20E945E3BC82FDD2751
:10743000C5FF1AC068E083E20E94773BC6FF10C018
:1074400020914C0130914D0180914E0190914F015E
:10745000281739072CF486E491E00E94893904C08A
:1074600061E087E20E94773BDF91CF91089588E049
:107470000E945E3B08958AE00E945E3B80FF03C04D
:107480000E94113A08958AE20E945E3B82E30E94C4
:107490005E3B8AE30E945E3B08958EE00E945E3B65
:1074A00008950F931F93CF93DF93CDB7DEB728973F
:1074B0000FB6F894DEBF0FBECDBF86E20E945E3BE2
:1074C00086FF79C08E010F5F1F4F80913A010E94A5
:1074D0005E3BF80181938F01CE010996E817F90709
:1074E000A1F78E010F5F1F4F68E087E20E94773B94
:1074F00068E083E20E94773B80E20E945E3B8F77E8
:10750000682F80E20E94773B898199279C01207631
:10751000307020323105B1F120343105B9F1232B1F
:10752000D9F58F719070892B19F5F801818186301A
:1075300051F0873018F48530B1F409C0893079F002
:107540008B3089F426C0C8010E94D3392DC060E475
:1075500080E20E94773B6B81605884E023C0C801C1
:107560000E947C3921C08BE890E00E94853B14C0CA
:1075700066E471E0C8010E94473886E491E00E9409
:10758000893912C0C8010E94493803C0C8010E944D
:10759000483865E083E206C080E20E945E3B805886
:1075A000682F80E20E94773BF80180818823D1F424
:1075B00065E083E215C020914E0130914F0180912A
:1075C0004A0190914B018217930764F410924F0186
:1075D00010924E0168E083E20E94773B61E087E20F
:1075E0000E94773B28960FB6F894DEBF0FBECDBF42
:1075F000DF91CF911F910F9108950F931F93CF9318
:10760000DF93CDB7DEB7C054D0400FB6F894DEBFDD
:107610000FBECDBF8CE00E945E3B992780FF03C068
:107620000E94513A27C081FF25C08EE20E945E3B36
:107630008DE20E945E3B89838E010F5F1F4F0F5FBB
:107640001F4F0E94523BF8018083CE01805C9F4F08
:1076500008171907A1F7E091AB00F091AC00CE013B
:107660000196099568E08FE20E94773B61E08FE226
:107670000E94773BC05CDF4F0FB6F894DEBF0FBEB1
:10768000CDBFDF91CF911F910F91089585B7826093
:1076900085BF8BB780648BBF88EF81BB82B3886363
:1076A00082BB089582B398E1892782BB0000000065
:1076B00082B3892782BB83B3992708959FEF94BB38
:1076C00085BB82B398E6892782BB82B3892782BBB8
:1076D000000014BA0E94523B9927089585BB82B3DB
:1076E00098E2892782BB82B3892782BB089585BB34
:1076F0008FEF84BB82B398E6892782BB82B3892748
:1077000082BB862F0E946E3B08950E941E3C089506
:107710009093B7008093B6007093B9006093B8005F
:1077200008959093AC008093AB0008951F9386E07A
:107730000E945E3B992786FF03C00E94FD3A0EC05F
:1077400082FF03C00E943B3A09C081FF03C00E9430
:10775000373A04C084FF02C00E944D3A87E00E947D
:107760005E3B182F60E087E00E94773B612F87E047
:107770000E94773B1F9108950E945B3961E080E091
:107780000E94773B80E00E945E3B80FDFBCF62E081
:1077900081E00E94773B60E18FE00E94773B60E8E8
:1077A00084E00E94773B60E480E20E94773B68E0DF
:1077B00083E20E94773B69E087E20E94773B6FE0BB
:1077C0008DE00E94773B6FE08BE00E94773B60E5A5
:1077D00089E00E94773B66ED87E00E94773B62E09C
:1077E00085E00E94773B6CEC80E00E94773B089537
:1077F00080EC8BB988E98AB986E880BD10BC8AE143
:1078000089B98CB15F99FDCF08955D9BFECF8CB98E
:1078100008955F9BFECF8CB1992708958A3310F4A9
:10782000805301C087556A3310F4605301C0675517
:107830008295807F6F70862B99270895FC0104C084
:107840005D9BFECF31968CB980818823C9F708955E
:10785000982F92959F708F709A3020F45D9BFECF89
:10786000905D03C05D9BFECF995A9CB98A3020F48D
:107870005D9BFECF805D03C05D9BFECF895A8CB9B6
:10788000089597FB092E07260AD077FD04D00CD067
:1078900006D000201AF4709561957F4F0895F6F791
:1078A000909581959F4F0895AA1BBB1B51E107C07E
:1078B000AA1FBB1FA617B70710F0A61BB70B881F80
:1078C000991F5A95A9F780959095BC01CD0108950F
:1078D000E199FECFBFBBAEBBE09A11960DB2089501
:1078E000E199FECFBFBBAEBB0DBA11960FB6F894AF
:0878F000E29AE19A0FBE08952F
:1078F80009021900010100A01A0904000002000091
:1079080000000705020240000012011001000000FB
:10791800088117620C000000000001756E73757015
:10792800706F72746564207374616E646172642030
:067938007265710A0D00EA
:040000030000700089
:00000001FF
